:100000000FC0000053C0000000000000000000000E
:1000100000000000000000000000000000000000E0
:100020000FED0DBF11272227AA27BB27C0E6DD272A
:10003000E0E0F2E003E00EBD00E002B903E309B93D
:1000400008E00AB90CE005BF00E80BBF002707BBBA
:1000500000E101BB0FEF08BB78940AD0FECF949A61
:100060004F934BB145FFFDCF4F914CB994980895F4
:1000700049EFF5DF46B74F70F2DF40916000EFDFE8
:1000800040916100ECDF40916200E9DF4091630044
:10009000E6DF40916400E3DF40916500E0DF4091DE
:1000A0006600DDDF40916700DADF0895C83612F0A0
:1000B000C0E6DD278CB59DB5C297C29749979923B5
:1000C00019F0C0E6DD2706C0E0E0F2E0E80FF91F16
:1000D000C895099200270DBD03950CBD1895000029
:1000E0000000000000000000000000000000000010
:1000F0000000000000000000000000000000000000
:1001000000000000000000000000000000000000EF
:1001100000000000000000000000000000000000DF
:1001200000000000000000000000000000000000CF
:1001300000000000000000000000000000000000BF
:1001400000000000000000000000000000000000AF
:10015000000000000000000000000000000000009F
:10016000000000000000000000000000000000008F
:10017000000000000000000000000000000000007F
:10018000000000000000000000000000000000006F
:10019000000000000000000000000000000000005F
:1001A000000000000000000000000000000000004F
:1001B000000000000000000000000000000000003F
:1001C000000000000000000000000000000000002F
:1001D000000000000000000000000000000000001F
:1001E000000000000000000000000000000000000F
:1001F00000000000000000000000000000000000FF
:1002000064656666676869696A6B6B6C6D6E6E6F54
:1002100070717172737374757676777879797A7B89
:100220007B7C7D7E7E7F80808182838384858686C1
:10023000878888898A8B8B8C8D8E8E8F90909192F7
:10024000939394959696979898999A9B9B9C9D9D2D
:100250009E9FA0A0A1A2A3A3A4A5A5A6A7A8A8A964
:10026000AAABABACADADAEAFB0B0B1B2B2B3B4B59A
:10027000B5B6B7B8B8B9BABABBBCBDBDBEBFC0C0D1
:10028000C1C2C2C3C4C5C5C6C7C8C8C8C8C8C8C813
:00000001FF
